:040000007EEF20F07F
:1000080000C016F001C015F0E1CF19F0E2CF1AF0E8
:10001800E9CF17F0EACF18F0F2A437D0F2AA35D01A
:100028008A86CD90D80E0001C16F000EC26F010EF6
:10003800C125E96E000EC221EA6EEECFCFFFC1C026
:10004800E9FFC2C0EAFFEECFCEFF9D809E908A8274
:10005800CD80DA0EC36F000EC46F010EC325E96EA2
:10006800000EC421EA6EEECFB3FFC3C0E9FFC4C0DF
:10007800EAFFEECFB2FFA082A1928A84B180F29407
:10008800630ED76EC00ED66E8A969EA005D09DA030
:1000980003D08A92CD909E90A1A205D0A0A203D0B1
:1000A8008A94B190A1929DAA75D09EAA73D0AECF22
:1000B800DEF0ABA40ED00001AB9E010EA525006EAC
:1000C800000EA621016E00C0A5F001C0A6F0AB8EFF
:1000D800DE6BABA20ED00001AB98010EB325006E0B
:1000E800000EB421016E00C0B3F001C0B4F0AB88BB
:1000F800DE6B0001DE510D0A3CE0DF0EDC25E16E0F
:10010800000EDD21E26EDEC0E6FFDCC0B5F0DDC02A
:10011800B6F0010EDC25006E000EDD21016E00C078
:10012800DCF001C0DDF0800E000A006E800EDD19E3
:10013800005C02E1DC514F0819E2020EB76F000EB5
:10014800B86F9D9A010EDC5D006E000EDD59016EE0
:10015800DF0E0024E16E000E0120E26EE66ADCC0CC
:10016800B5F0DDC0B6F0DC6BDD6B02D0B76BB86BF9
:1001780011D0DF0EDC25E16E000EDD21E26EE66AAD
:10018800010EB76F000EB86FDCC0B5F0DDC0B6F079
:10019800DC6BDD6B16C000F015C001F017C0E9FF7D
:0E01A80018C0EAFF19C0E1FF1AC0E2FF110003
:1001B6000B820BAEE5EF00F0036802680168006889
:0801C6000A360232FF0E12009E
:0E01CE00026A016A006A086A036A000E1200E3
:1001DC000B840BAEF9EF00F0010E036E026A016A9C
:0A01EC00006A0A360232FF0E12000C
:0801F6000AAE029E000E120089
:1001FE000CB041EF01F00CA2E7EF01F00E6A000E19
:10020E00026458EF01F0F00E0214D8A423EF01F0AF
:10021E00023A01380F0B02260138F00B016E00383E
:10022E000F0B01260038F00B006E08380F0B00265E
:10023E000838F00B086E0E84D89002BE3CEF01F029
:10024E0008360036013602360E2A02BE3CEF01F0A9
:10025E0008360036013602360E2A02BE3CEF01F099
:10026E0008360036013602360E2A0E500364DDEFD4
:10027E0001F0035E0BBC08AEE2EF01F0D880800EF9
:10028E0008640030000E002201220222D8A0E2EF04
:10029E0001F0023201320032034AE7EF01F0E2EFE1
:1002AE0001F001C002F000C001F008C000F0086AC1
:1002BE00000E0E8602648FEF01F0F00E0214D8A429
:1002CE0077EF01F0023A01380F0B02260138F00BDE
:1002DE00016E00380F0B01260038F00B006E0E84F5
:1002EE00D89002BE3CEF01F00036013602360E2ADF
:1002FE0002BE3CEF01F00036013602360E2A02BE77
:10030E003CEF01F00036013602360E2A3CEF01F0CA
:10031E0001C002F000C001F0006A000E0E960E88B9
:10032E000264BCEF01F0F00E0214D8A4A7EF01F0A6
:10033E00023A01380F0B02260138F00B016E0E84C3
:10034E00D89002BE3CEF01F0013602360E2A02BEF4
:10035E003CEF01F0013602360E2A02BE3CEF01F0F0
:10036E00013602360E2A3CEF01F001C002F0016A9E
:10037E00000E0E860264ECEF01F0F00E0214D8A40B
:10038E00CBEF01F0023A0E84D89002BE3CEF01F0A2
:10039E0002360E2A02BE3CEF01F002360E2A02BED3
:1003AE003CEF01F002360E2A3CEF01F0010E0C6E0E
:1003BE000EDFEFEF01F0020E0C6E16DFEFEF01F025
:1003CE00040E0C6EF1DEEFEF01F0080E0C6EF8DE8F
:0203DE0012000B
:0803E0000B6A0B86FF0E1200F0
:1003E800086A096A000E0762036479EF02F0025096
:1003F80006180A6E075003267E0ED8A00AEF02F0F0
:10040800035ED8B07DEF02F00EEF02F0035ED8A0D5
:1004180081EF02F0028E068E02C00EF001C00BF0D2
:1004280000C00DF000500402F4CF0CF0015005029A
:10043800F4CF00F0F3CF08F00402F3500C26F45088
:100448000822000E00220D500502F3500C26F4502D
:100458000822000E002202500402F3500826F4502D
:10046800002202500502016A000E0122F350002604
:10047800F45001220D500602F3500826F4500022D1
:10048800026A000E012202220B500602F3500026D7
:10049800F4500122000E02220E500602F3500126EB
:1004A800F450022202BE61EF02F00836003601362F
:1004B80002360306D8B481EF02F074EF02F0D88058
:1004C800800E08640030000E002201220222D8A00B
:1004D80074EF02F0023201320032034A7DEF02F07B
:1004E8000AAE029E000E83EF02F0010E6CDE83EF6F
:1004F80002F0020E5CDE83EF02F0040E6BDE1200E7
:100508000D6A086A0050D8B4000C04180A6E0ABEB6
:100518000D1E0B6A04AE02D0041E042A00AE02D0DF
:10052800001E002A005004100A6E0ABE1FD0045094
:10053800085E003600340836045008260036060ED9
:100548000C6E00340836045000B0085E00A008267F
:1005580000360C2EF6D700A008260BB015D00DAE2D
:10056800000C001E002A081E082A000C04AE09D040
:1005780000BE04D00050086E006AF1D7006A002A55
:10058800000C001E0B2AD3D7082A0450085CD8A4F4
:0E059800E6D7086A002A00AEE2D7FF0C120078
:1005A600025006180E6E086A096A0B6A0350076441
:1005B600C6EF03F006500A6E068E028E03500B6ECF
:1005C6000750036E000E0B6416EF03F00B50075E28
:1005D600D8B4B7EF03F0070E076485EF03F0075EA4
:1005E60000C008F001C000F002C001F0026A074E28
:1005F600B7EF03F007645AEF03F0075E00C008F098
:1006060001C000F0016A074EB7EF03F0076438EF48
:1006160003F0075E00C008F0006A074EB7EF03F06C
:1006260007641FEF03F00AC002F005C001F004C022
:1006360000F0086AE1EF04F0030E07642AEF03F006
:10064600075E08380F0B086E074EB7EF03F0D89019
:100656000832074EB7EF03F0D8900832074EB7EFCF
:1006660003F0D8900832B7EF03F0030E076449EFA2
:1006760003F0075E08380F0B086E0038F00B0826EB
:1006860000380F0B006E074EB7EF03F0D89000321C
:100696000832074EB7EF03F0D89000320832074E03
:1006A600B7EF03F0D89000320832B7EF03F0030E2D
:1006B600076471EF03F0075E08380F0B086E003809
:1006C600F00B082600380F0B006E0138F00B0026E1
:1006D60001380F0B016E074EB7EF03F0D8900132C9
:1006E60000320832074EB7EF03F0D89001320032DD
:1006F6000832074EB7EF03F0D890013200320832C5
:10070600B7EF03F0030E0764A2EF03F0075E0838A5
:100716000F0B086E0038F00B082600380F0B006E22
:100726000138F00B002601380F0B016E0238F00B72
:10073600012602380F0B026E074EB7EF03F0D89072
:100746000232013200320832074EB7EF03F0D8907A
:100756000232013200320832074EB7EF03F0D8906A
:100766000232013200320832096A000E0EAEABEFD9
:1007760004F0081E001E011E021E082A0022012285
:100786000222ABEF04F00750D8A4CCEF03F0E1EF60
:1007960004F0096A02C00AF0028E068E0750035C56
:1007A600076ED8B49EEF04F0070E07646CEF04F0F2
:1007B600075E0450096E0550046E0650056E066A03
:1007C600074E9EEF04F0070E076441EF04F0075E44
:1007D6000450096E0550046E056A074E9EEF04F03C
:1007E600070E07641FEF04F0075E0450096E046AE3
:1007F600074E9EEF04F0070E076406EF04F00AC0EA
:1008060002F0E1EF04F0030E076411EF04F0075E57
:1008160009380F0B096E074E9EEF04F0D890093287
:10082600074E9EEF04F0D8900932074E9EEF04F073
:10083600D89009329EEF04F0030E076430EF04F0FF
:10084600075E09380F0B096E0438F00B09260438C9
:100856000F0B046E074E9EEF04F0D8900432093257
:10086600074E9EEF04F0D89004320932074E9EEFF1
:1008760004F0D890043209329EEF04F0030E0764A8
:1008860058EF04F0075E09380F0B096E0438F00BB9
:10089600092604380F0B046E0538F00B04260538BC
:1008A6000F0B056E074E9EEF04F0D890053204320A
:1008B6000932074E9EEF04F0D89005320432093211
:1008C600074E9EEF04F0D8900532043209329EEFAF
:1008D60004F0030E076489EF04F0075E09380F0B76
:1008E600096E0438F00B092604380F0B046E053820
:1008F600F00B042605380F0B056E0638F00B05269F
:1009060006380F0B066E074E9EEF04F0D89006329F
:10091600053204320932074E9EEF04F0D8900632B3
:10092600053204320932074E9EEF04F0D8900632A3
:10093600053204320932086A000E0EAEABEF04F03F
:10094600091E041E051E061E092A04220522062269
:1009560009500826045000220550012206500222A2
:100966000EBEC2EF04F0D8A0D1EF04F0023201327D
:1009760000320832033ED1EF04F0DBEF04F0D8B0CA
:10098600D6EF04F0000E081E001E011E021E082AE5
:100996000022012202220A7ED6EF04F0010E0C6E1E
:1009A6002BDCE3EF04F0020E0C6E26DCE3EF04F022
:1009B600040E0C6EDBEC00F0E3EF04F0000E0C6EA0
:0209C60012001D
:1009C800086A080E0C6E003408360450085ED8B069
:0E09D80002D00826D89000360C2EF5D712005B
:1009E6000B800BAEFFEF04F0026A0AAEFF0E026E3A
:0C09F600016E006E0A360232FF0E120085
:100A02000134083609360450085E0550D8A0053C6A
:100A1200095E003601360F0E0C6E013408360936B7
:100A2200045000A006D0085E0550D8A0053C095E1F
:100A320005D008260550D8B0053C092600360136F7
:100A42000C2EEBD700B006D0045008260550D8B0C3
:080A5200053C0926000012001A
:100A5A000B6A0C6A086A0350D8B4B1EF05F002C0F9
:100A6A000AF0028E9E0E035E03AEA1EF05F0036C40
:100A7A00080E035CD8A06EEF05F0036E083600C0BE
:100A8A0008F001C000F002C001F0026A080E035C1F
:100A9A00D8A06EEF05F0036E083600C008F001C05A
:100AAA0000F0016A080E035CD8A06EEF05F0036E31
:100ABA00083600C008F0006A080E035CD8A06EEF82
:100ACA0005F0036E0836086A0350D8A4D8907AEF66
:100ADA0005F00350D8B47AEF05F0D890023201320B
:100AEA0000320832032E72EF05F00BBC08A08BEF20
:100AFA0005F0D8A08BEF05F0082AD8B4002AD8B49C
:100B0A00012AD8B4022A02BEB5EF05F00AAEB1EF47
:100B1A0005F0021E011E001E081E082AD8B4002A6B
:100B2A00D8B4012AD8B4022AB1EF05F0026A016AE0
:100B3A00006A086AB1EF05F00B800BAEBBEF05F057
:100B4A00026A0AAEBBEF05F0026E016E006E086E15
:100B5A000A360232BBEF05F00C6A000EBCEF05F054
:100B6A00010E0C6E000E3ADFBCEF05F0FF0E0250CC
:100B7A00036E0150026E0050016E0850006E1200A2
:100B8A000050086E0150006E0250016E0350026E52
:100B9A00036A0B6A0C6A9E0E036E0A6A020E0C6ED8
:060BAA00FFEC00F0120058
:100BB0000B6A0A6A096A00500402F4CF09F0F3CF05
:100BC00008F001500502F4CF0BF0F3CF0AF000500B
:100BD0000502F3500926F4500A22E86A0B2201505C
:100BE0000402F3500926F4500A22E86A0B2208C0D6
:100BF00000F009C001F00AC002F00BC003F01200BF
:100C00000B6A0A6A096A086A0E6A033408360450D5
:100C1000085E0550D8A0053C095E0650D8A0063CE9
:100C20000A5E0750D8A0073C0B5EE86AD8A0010E08
:100C30000E5E0336070E0C6E0334083609360A368C
:100C40000B360E36045003A012D0085E0550D8A013
:100C5000053C095E0650D8A0063C0A5E0750D8A0A5
:100C6000073C0B5EE86AD8A0010E0E5E11D0082684
:100C70000550D8B0053C09260650D8B0063C0A26D7
:100C80000750D8B0073C0B26E86AD8B0010E0E26F4
:100C900003360C2ED1D70234083609360A360B3605
:100CA0000E36045003A012D0085E0550D8A0053CB3
:100CB000095E0650D8A0063C0A5E0750D8A0073C43
:100CC0000B5EE86AD8A0010E0E5E11D00826055012
:100CD000D8B0053C09260650D8B0063C0A26075075
:100CE000D8B0073C0B26E86AD8B0010E0E260236B3
:100CF000070E0C6E0234083609360A360B360E36ED
:100D0000045002A012D0085E0550D8A0053C095E30
:100D10000650D8A0063C0A5E0750D8A0073C0B5EE0
:100D2000E86AD8A0010E0E5E11D008260550D8B092
:100D3000053C09260650D8B0063C0A260750D8B014
:100D4000073C0B26E86AD8B0010E0E2602360C2EA0
:100D5000D1D70134083609360A360B360E36045020
:100D600002A012D0085E0550D8A0053C095E0650CE
:100D7000D8A0063C0A5E0750D8A0073C0B5EE86A84
:100D8000D8A0010E0E5E11D008260550D8B0053C43
:100D900009260650D8B0063C0A260750D8B0073CB2
:100DA0000B26E86AD8B0010E0E260136070E0C6E2F
:100DB0000134083609360A360B360E36045001A0C7
:100DC00012D0085E0550D8A0053C095E0650D8A098
:100DD000063C0A5E0750D8A0073C0B5EE86AD8A024
:100DE000010E0E5E11D008260550D8B0053C09262C
:100DF0000650D8B0063C0A260750D8B0073C0B2650
:100E0000E86AD8B0010E0E2601360C2ED1D7003478
:100E1000083609360A360B360E36045001A012D0B9
:100E2000085E0550D8A0053C095E0650D8A0063CD7
:100E30000A5E0750D8A0073C0B5EE86AD8A0010EF6
:100E40000E5E11D008260550D8B0053C0926065084
:100E5000D8B0063C0A260750D8B0073C0B26E86AF3
:100E6000D8B0010E0E260036070E0C6E0034083680
:100E700009360A360B360E36045000A012D0085E32
:100E80000550D8A0053C095E0650D8A0063C0A5E75
:100E90000750D8A0073C0B5EE86AD8A0010E0E5E92
:100EA00011D008260550D8B0053C09260650D8B008
:100EB000063C0A260750D8B0073C0B26E86AD8B093
:100EC000010E0E2600360C2ED1D700B00ED00450E5
:100ED00008260550D8B0053C09260650D8B0063C77
:0C0EE0000A260750D8B0073C0B26120071
:100EEC006E0E01016A5DD8A0C6D0640E046E6AC194
:100EFC0000F064DD120E0024056E066A000E062258
:100F0C0005C000F006C001F0000E06BEFF0E026E1A
:100F1C00036E003600900136023603360036009020
:100F2C00013602360336360E0024F66E480E0120CA
:100F3C00F76E000E0220F86E0900F5CF00F00900E4
:100F4C00F5CF01F00900F5CF02F00900F5CF03F061
:100F5C00000E046E000E056E000E066E7E0E076E01
:100F6C00F4EC01F000C06BF101C06CF102C06DF14A
:100F7C0003C06EF1640E046E6AC100F01FDD08C080
:100F8C0000F00A0E046E1ADD090E0024056E066AC6
:100F9C00000E062205C000F006C001F0000E06BED1
:100FAC00FF0E026E036E00360090013602360336D9
:100FBC0000360090013602360336360E0024F66EEB
:100FCC00480E0120F76E000E0220F86E0900F5CFD6
:100FDC0000F00900F5CF01F00900F5CF02F009008F
:100FEC00F5CF03F06BC104F06CC105F06DC106F0D8
:100FFC006EC107F0F4EC01F000C06BF101C06CF1B4
:10100C0002C06DF103C06EF10A0E046E6AC100F0ED
:10101C00D5DC08C000F000C001F0000E026E036EBB
:10102C00046E013601900236033604360136019007
:10103C00023603360436360E0124F66E480E0220B4
:10104C00F76E000E0320F86E0900F5CF00F00900D2
:10105C00F5CF01F00900F5CF02F00900F5CF03F050
:10106C006BC104F06CC105F06DC106F06EC107F0E8
:10107C00F4EC01F0AFD06A510A08D8B07CD00A0E5B
:10108C00046E6AC100F09ADC090E0024056E066A33
:10109C00000E062205C000F006C001F0000E06BED0
:1010AC00FF0E026E036E00360090013602360336D8
:1010BC0000360090013602360336360E0024F66EEA
:1010CC00480E0120F76E000E0220F86E0900F5CFD5
:1010DC0000F00900F5CF01F00900F5CF02F009008E
:1010EC00F5CF03F0000E046E000E056E000E066EBA
:1010FC007E0E076EF4EC01F000C06BF101C06CF1D8
:10110C0002C06DF103C06EF10A0E046E6AC100F0EC
:10111C0055DC08C000F000C001F0000E026E036E3A
:10112C00046E013601900236033604360136019006
:10113C00023603360436360E0124F66E480E0220B3
:10114C00F76E000E0320F86E0900F5CF00F00900D1
:10115C00F5CF01F00900F5CF02F00900F5CF03F04F
:10116C006BC104F06CC105F06DC106F06EC107F0E7
:10117C00F4EC01F02FD06AC100F0000E016E026E8B
:10118C00036E0036009001360236033600360090AE
:10119C00013602360336360E0024F66E480E012058
:1011AC00F76E000E0220F86E0900F5CF00F0090072
:1011BC00F5CF01F00900F5CF02F00900F5CF03F0EF
:1011CC00000E046E000E056E000E066E7E0E076E8F
:0611DC00F4EC01F012002A
:1011E2000A6A0350D8A40A800750D8A40A820A5077
:1011F200D8B454EF09F0030AD8B40DEF09F00AB0DD
:1012020008EF09F006AE52EF09F050EF09F002AE16
:1012120050EF09F052EF09F00250800B0A6E029E65
:101222000650800B069E0A18D8B41EEF09F00A5029
:10123200D8B450EF09F052EF09F00750035CD8B46C
:1012420028EF09F0D8A044EF09F04AEF09F0065060
:10125200025CD8B432EF09F0D8A044EF09F04AEFAB
:1012620009F00550015CD8B43CEF09F0D8A044EF76
:1012720009F04AEF09F00450005CD8B454EF09F0C9
:10128200D8B04AEF09F00A52D8B452EF09F050EF41
:1012920009F00A52D8B450EF09F052EF09F0D880A1
:0E12A2001200D8901200D880D88412001200DA
:1012B0000450000A08E10550000A05E1FF0E006E27
:1012C0007F0E016E58D00D6A096A086A015000103D
:1012D000D8B4000C015005180A6E0ABE0D1E0B6A28
:1012E00005AE05D0041E051E042AD8B4052A01AE99
:1012F00005D0001E011E002AD8B4012A0150051095
:101300000A6E0ABE10D001EC05F00BB020D00DAE75
:10131000000C001E011E002AD8B4012A081E091E56
:10132000082AD8B4092A000C05AE0DD001BE07D09A
:101330000150096E0050086E016A006AE8D7016A20
:10134000006A002A000C011E001E0B2ADDD7082AA5
:10135000D8B4092A0450085CD8A4D9D70550095C30
:10136000D8A4D5D7096A086A002AD8B4012A01AEE0
:08137000CED70000FF0C1200B3
:10137800800E01016A19006E800E000A005CD8B068
:101388006DD16A510008016E01C06AF1800E011822
:10139800006E800E6E0A005CD8A0C0D0640E046E89
:1013A8006AC100F084EC02F0120E0024056E000EF3
:1013B80000BEFF0E066E000E062205C000F006C035
:1013C80001F0000E06BEFF0E026E036E003600909E
:1013D80001360236033600360090013602360336EF
:1013E800360E0024F66E480E0120F76E000E02201D
:1013F800F86E0900F5CF6BF10900F5CF6CF1090023
:10140800F5CF6DF10900F5CF6EF1640E046E6AC177
:1014180000F084EC02F008C000F00A0E046E84ECC0
:1014280002F0090E0024056E000E00BEFF0E066EC7
:10143800000E062205C000F006C001F0000E06BE30
:10144800FF0E026E036E0036009001360236033638
:1014580000360090013602360336360E0024F66E4A
:10146800480E0120F76E000E0220F86E0900F5CF35
:1014780000F00900F5CF01F00900F5CF02F00900EE
:10148800F5CF03F06BC104F06CC105F06DC106F037
:101498006EC107F0F4EC01F000C06BF101C06CF113
:1014A80002C06DF103C06EF10A0E046E6AC100F04D
:1014B80084EC02F008C000F000C001F0000E00BE8D
:1014C800FF0E026E036E046E01360190023603367B
:1014D800043601360190023603360436360E0124EE
:1014E800F66E480E0220F76E000E0320F86E090013
:1014F800F5CF00F00900F5CF01F00900F5CF02F0B3
:101508000900F5CF03F06BC104F06CC105F06DC1A3
:1015180006F06EC107F0F4EC01F007D2800E0A0A5B
:10152800006E800E6A19005C71E20A0E046E6AC1D0
:1015380000F084EC02F0090E0024056E000E00BED7
:10154800FF0E066E000E062205C000F006C001F070
:10155800000E06BEFF0E026E036E003600900136C6
:101568000236033600360090013602360336360E50
:101578000024F66E480E0120F76E000E0220F86E69
:101588000900F5CF6BF10900F5CF6CF10900F5CF33
:101598006DF10900F5CF6EF10A0E046E6AC100F014
:1015A80084EC02F008C000F000C001F0000E00BE9C
:1015B800FF0E026E036E046E01360190023603368A
:1015C800043601360190023603360436360E0124FD
:1015D800F66E480E0220F76E000E0320F86E090022
:1015E800F5CF00F00900F5CF01F00900F5CF02F0C2
:1015F8000900F5CF03F06BC104F06CC105F06DC1B3
:1016080006F06EC107F0F4EC01F08FD16AC100F06A
:10161800000E6ABFFF0E016E026E036E0036009068
:10162800013602360336003600900136023603369C
:10163800360E0024F66E480E0120F76E000E0220CA
:10164800F86E0900F5CF00F00900F5CF01F00900A8
:10165800F5CF02F00900F5CF03F067D1800E6A19C3
:10166800006E800E6E0A005CD8A0C0D0640E046EB6
:101678006AC100F084EC02F0120E0024056E000E20
:1016880000BEFF0E066E000E062205C000F006C062
:1016980001F0000E06BEFF0E026E036E00360090CB
:1016A800013602360336003600900136023603361C
:1016B800020E0024F66E480E0120F76E000E02207E
:1016C800F86E0900F5CF6BF10900F5CF6CF1090050
:1016D800F5CF6DF10900F5CF6EF1640E046E6AC1A5
:1016E80000F084EC02F008C000F00A0E046E84ECEE
:1016F80002F0090E0024056E000E00BEFF0E066EF5
:10170800000E062205C000F006C001F0000E06BE5D
:10171800FF0E026E036E0036009001360236033665
:1017280000360090013602360336020E0024F66EAB
:10173800480E0120F76E000E0220F86E0900F5CF62
:1017480000F00900F5CF01F00900F5CF02F009001B
:10175800F5CF03F06BC104F06CC105F06DC106F064
:101768006EC107F0F4EC01F000C06BF101C06CF140
:1017780002C06DF103C06EF10A0E046E6AC100F07A
:1017880084EC02F008C000F000C001F0000E00BEBA
:10179800FF0E026E036E046E0136019002360336A8
:1017A800043601360190023603360436020E01244F
:1017B800F66E480E0220F76E000E0320F86E090040
:1017C800F5CF00F00900F5CF01F00900F5CF02F0E0
:1017D8000900F5CF03F06BC104F06CC105F06DC1D1
:1017E80006F06EC107F0F4EC01F09FD0800E0A0AF3
:1017F800006E800E6A19005C71E20A0E046E6AC1FE
:1018080000F084EC02F0090E0024056E000E00BE04
:10181800FF0E066E000E062205C000F006C001F09D
:10182800000E06BEFF0E026E036E003600900136F3
:101838000236033600360090013602360336020EB1
:101848000024F66E480E0120F76E000E0220F86E96
:101858000900F5CF6BF10900F5CF6CF10900F5CF60
:101868006DF10900F5CF6EF10A0E046E6AC100F041
:1018780084EC02F008C000F000C001F0000E00BEC9
:10188800FF0E026E036E046E0136019002360336B7
:10189800043601360190023603360436020E01245E
:1018A800F66E480E0220F76E000E0320F86E09004F
:1018B800F5CF00F00900F5CF01F00900F5CF02F0EF
:1018C8000900F5CF03F06BC104F06CC105F06DC1E0
:1018D80006F06EC107F0F4EC01F027D06AC100F001
:1018E800000E6ABFFF0E016E026E036E0036009096
:1018F80001360236033600360090013602360336CA
:10190800020E0024F66E480E0120F76E000E02202B
:10191800F86E0900F5CF00F00900F5CF01F00900D5
:0C192800F5CF02F00900F5CF03F012002B
:101934000450000A12E10550000A0FE10650000AA3
:101944000CE10750000A09E1FF0E006EFF0E016E64
:101954007F0E026EFF0E036EA8D0086A096A075054
:10196400D8B445EF0DF00350D8B44AEF0DF002504F
:1019740006180A6E028E068E0E6A02C008F001C0B6
:101984000CF000C00DF004500D5E0550D8A0053CCD
:101994000C5E0650D8A0063C085E086A0C6A0D6A04
:1019A400D8A0DCEF0CF0D8900232013200320832B9
:1019B400010E0E6E0750035ED8A0E9EF0CF07E0E08
:1019C4000E240326D8B04FEF0DF0EFEF0CF07E0E8F
:1019D4000E240326D8A054EF0DF0180E0B6E0D360E
:1019E4000C3608360036013602360E360450005ED8
:1019F4000550D8A0053C015E0650D8A0063C025E06
:101A040006340E120EA00AEF0DF00D8015EF0DF046
:101A1400045000260550D8B0053C01260650D8B025
:101A2400062802260D900B2EF1EF0CF03BEF0DF083
:101A3400D8900036013602360E360450005E05504A
:101A4400D8A0053C015E0650D8A0063C025E0634D0
:101A54000E10010B0D26D8B00C2AD8B4082AD8A42D
:101A64003BEF0DF008320C320D32032AD8B44FEF9D
:101A74000DF00AAE089E0850026E0C50016E0D5017
:101A8400006E57EF0DF0010EF0EC01F057EF0DF082
:101A9400020EE7EC00F057EF0DF0040EDBEC00F063
:0C1AA40057EF0DF0080EEEEC00F0120001
:101AB0000B6A0C6A0A6A086A0350D8B4E0EF0DF0AA
:101AC000028E9E0E035E03BE6BEF0DF0D8B46BEF7B
:101AD0000DF0D0EF0DF0036C080E035CD8A09DEF65
:101AE0000DF0036E083600C008F001C000F002C01F
:101AF00001F0026A080E035CD8A09DEF0DF0036EA2
:101B0000083600C008F001C000F0016A080E035C4E
:101B1000D8A09DEF0DF0036E083600C008F0006AF3
:101B2000080E035CD8A09DEF0DF0036E0836086A1E
:101B30000350D8A4D890A9EF0DF00350D8B4A9EF62
:101B40000DF0D8900232013200320832032EA1EF9C
:101B50000DF00BBC08A0BAEF0DF0D8A0BAEF0DF055
:101B6000082AD8B4002AD8B4012AD8B4022A02BE5E
:101B7000E4EF0DF00AAEE0EF0DF0021E011E001EB4
:101B8000081E082AD8B4002AD8B4012AD8B4022AD8
:101B9000E0EF0DF0026A016A006A086AE0EF0DF0FA
:101BA0000B800BAEEAEF0DF0026A0AAEEAEF0DF021
:101BB000026E016E006E086E0A360232EAEF0DF018
:101BC000000E0C6AEBEF0DF0010E0C6EF3EC04F05E
:101BD000EBEF0DF0FF0E0250036E0150026E00504D
:081BE000016E0850006E1200B6
:101BE80003500718D8A408EF0EF002500618D8A41E
:101BF80008EF0EF001500518D8A408EF0EF00050B9
:0E1C08000418D8B4D8841200D8941200120028
:081C1600067ED3EC02F012007F
:101C1E0001016A51390806E3300E6A5D03E3010ED5
:081C2E00006E01D0006A1200F3
:101C36000101626B636B566B576B44C100F045C183
:101C460001F046C102F0010E4427000E452346234B
:101C560000C0F6FF01C0F7FF02C0F8FF0900F5CF8C
:101C660000F000C053F10052D8B425EF1EF05351D6
:101C7600250A0BE042C1E1FF43C1E2FF53C1E6FF83
:101C8600424B432B624B632BD8D7546B556B566B29
:101C9600576B23D05687010E4427000E4523462353
:101CA60059D05681010E4427000E4523462352D0B3
:101CB6005683010E4427000E452346234BD05787F3
:101CC600010E4427000E4523462344D05685010EB7
:101CD6004427000E452346233DD044C1F6FF45C1A7
:101CE600F7FF46C1F8FF0900F5CF01F001502D0AB4
:101CF600D1E044C1F6FF45C1F7FF46C1F8FF090030
:101D0600F5CF01F00150200ACCE044C1F6FF45C1F1
:101D1600F7FF46C1F8FF0900F5CF01F001502B0A85
:101D2600C7E044C1F6FF45C1F7FF46C1F8FF090009
:101D3600F5CF01F00150230AC2E044C1F6FF45C1C8
:101D4600F7FF46C1F8FF0900F5CF01F00150300A50
:101D5600BDE001D09ED756A301D0569156A701D01B
:101D6600569544C1F6FF45C1F7FF46C1F8FF090085
:101D7600F5CF00F0000E016E00C06AF14DDF005293
:101D860035E0546B556B54C100F055C101F00A0E95
:101D9600046E000E056ED8EC05F044C1F6FF45C191
:101DA600F7FF46C1F8FF0900F5CF02F00250002404
:101DB600546F000E0120556F300E545F000E555BB8
:101DC600010E4427000E4523462344C1F6FF45C1B4
:101DD600F7FF46C1F8FF0900F5CF00F0000E016ECF
:101DE60000C06AF119DF0052CEE133D044C1F6FFDC
:101DF60045C1F7FF46C1F8FF0900F5CF01F00150D4
:101E06002A0A27E147C1E9FF48C1EAFFEECF00F001
:101E1600EECF01F000C0E9FF01C0EAFFEECF54F1BA
:101E2600EECF55F147C1E9FF48C1EAFF020EEE24A5
:101E3600006E000EEE20016E47C1E1FF48C1E2FFD1
:101E460000C0E6FF01C0E6FF010E4427000E452351
:101E5600462344C1F6FF45C1F7FF46C1F8FF090016
:101E6600F5CF01F001502E0A6FE1010E4427000E56
:101E76004523462344C1F6FF45C1F7FF46C1F8FF97
:101E86000900F5CF01F001502A0A28E147C1E9FF10
:101E960048C1EAFFEECF00F0EECF01F000C0E9FF47
:101EA60001C0EAFFEECF51F1EECF52F147C1E9FF93
:101EB60048C1EAFF020EEE24006E000EEE20016E0F
:101EC60047C1E1FF48C1E2FF00C0E6FF01C0E6FFEF
:101ED600010E4427000E4523462335D0516B526B25
:101EE60044C1F6FF45C1F7FF46C1F8FF0900F5CF2B
:101EF60000F0000E016E00C06AF18EDE005223E093
:101F060051C100F052C101F00A0E046E000E056EBA
:101F1600D8EC05F044C1F6FF45C1F7FF46C1F8FF0E
:101F26000900F5CF02F002500024516F000E012087
:101F3600526F300E515F000E525B010E4427000EA9
:101F460045234623CDD703D0516B526B578944C1E5
:101F560000F045C101F046C102F0010E4427000E13
:101F66004523462300C0F6FF01C0F7FF02C0F8FF75
:101F76000900F5CF53F1F9D062C100F063C101F059
:101F860029EF1EF05689E3D757852ED1568B5781F8
:101F96002BD1578329D1568D27D126D1568B568FD3
:101FA60023D147C1E9FF48C1EAFFEECF00F0EECFEB
:101FB60001F000C0E9FF01C0EAFFEECF5EF1EECF0F
:101FC6005FF147C1E9FF48C1EAFF020EEE24006E49
:101FD600000EEE20016E47C1E1FF48C1E2FF00C0DE
:101FE600E6FF01C0E6FF000E5F1902E1000E5E1972
:101FF60004E13C0E5E6F000E5F6F606B616B6051BB
:102006005E25E96E61515F21EA6EEE520BE0010E2C
:102016006025006E000E6121016E00C060F101C0F6
:1020260061F1EDD7515152110AE06151525D02E161
:102036006051515D04E251C160F152C161F15551E7
:10204600615D02E15451605D05E26051545F61518A
:10205600555B02D0546B556B56B716D054C100F081
:1020660055C101F0010E545F000E555B0050011082
:102076000BE042C1E1FF43C1E2FF200EE66E424B98
:10208600432B624B632BEAD760C102F061C103F0B8
:10209600010E605D006E000E6159016E00C060F1B8
:1020A60001C061F10250031019E05EC1E9FF5FC192
:1020B600EAFF42C1E1FF43C1E2FFEECFE6FF424B3A
:1020C600432B010E5E25006E000E5F21016E00C0DF
:1020D6005EF101C05FF1624B632BD6D756A716D0CF
:1020E60054C100F055C101F0010E545F000E555B5E
:1020F600005001100BE042C1E1FF43C1E2FF200E98
:10210600E66E424B432B624B632BEAD796D547C10B
:10211600E9FF48C1EAFFEECF00F0EECF01F000C0C4
:10212600E9FF01C0EAFFEECF53F147C1E9FF48C11D
:10213600EAFF020EEE24006E000EEE20016E47C18D
:10214600E1FF48C1E2FF00C0E6FF01C0E6FF530E13
:102156005E6F010E5F6F010E606F000E616F62D7DA
:10216600C00E5613000E57133FD05351000AD8B471
:1021760003D753516C0AD8B405D753514C0AD8B477
:1021860001D75351660AD8B4FFD65351450AD8B47D
:10219600FDD65351650AD8B4FAD65351670AD8B456
:1021A600F8D653516F0AD8B4F6D65351640AD8B448
:1021B600F4D65351690AD8B4F0D65351700AD8B43C
:1021C600EDD65351580AD8B4E9D65351780AD8B443
:1021D600E6D65351730AD8B4E4D65351630A97E04E
:1021E6005351750ABDE0B3D7000E5615006E575110
:1021F600070B016E00500110D8B4CCEF19F057A9A7
:1022060004D0060E516F000E526F47C1E9FF48C158
:10221600EAFFEECF00F0EECF01F000C0E9FF01C00B
:10222600EAFFEECF58F1EECF59F1EECF5AF1EECFED
:102236005BF147C1E9FF48C1EAFF040EEE24006ED8
:10224600000EEE20016E47C1E1FF48C1E2FF00C06B
:10225600E6FF01C0E6FF046A056A066A076A58C116
:1022660000F059C101F05AC102F05BC103F0F1EC74
:1022760008F0010ED8B0000E006E005205E05A7F3D
:10228600030E5613000E57135C6B5D6B58C100F0BE
:1022960059C101F05AC102F05BC103F0046A056A34
:1022A600066A076A9EDC000ED8A4010E006E005274
:1022B600D8B48AD05BC100F0016A026A036AFF0ED5
:1022C6000016000E01167E0E005E000E015A00C0BA
:1022D6005CF101C05DF1010E005E000E015A00C006
:1022E6005CF101C05DF1030E046E000E056ED8ECC4
:1022F60005F000C05CF101C05DF10A0E046E000E2F
:10230600056E58EC09F000C05CF101C05DF1800E6D
:102316000118026E800E025C02E1000E005C05E20E
:10232600010E01015C5F000E5D5B01015C5100085E
:102336006A6FBCEC09F058C104F059C105F05AC1E6
:1023460006F05BC107F0F4EC01F000C05EF101C0DD
:102356005FF102C060F103C061F1000E046E000E71
:10236600056E000E066E7F0E076E5EC100F05FC141
:1023760001F060C102F061C103F0F1EC08F0010E5A
:10238600D8B0000E006E005205E0010E5C5F000E34
:102396005D5B1AD0000E046E000E056E200E066EF2
:1023A600820E076E5EC100F05FC101F060C102F0EF
:1023B60061C103F0F1EC08F0000ED8B0010E006E1A
:1023C600005202E05C4B5D2B800E006E800E5D19A4
:1023D600005C02E15C51000803E3010E536F02D07A
:1023E6005CC153F157B118D057A315D0800E5D19B3
:1023F600006E7F0E005C02E1FC0E5C5D0BE3800E5E
:102406005D19006E800E5219005C02E151515C5D4F
:1024160001E201D001D0EFD35151521106E057A38A
:1024260004D0010E515F000E525B5251000802E1CA
:102436005151080803E2080E536F02D051C153F1FF
:1024460058C100F059C101F05AC102F05BC103F056
:10245600046A056A066A076AF4EC0DF0000ED8A451
:10246600010E006E0052D8B44BD15CC16AF1BCECCF
:1024760009F000C004F001C005F002C006F003C078
:1024860007F058C100F059C101F05AC102F05BC112
:1024960003F09AEC0CF000C058F101C059F102C0EB
:1024A6005AF103C05BF10101535100086A6FBCEC9D
:1024B60009F000C004F001C005F002C006F003C038
:1024C60007F058C100F059C101F05AC102F05BC1D2
:1024D60003F09AEC0CF000C064F101C065F102C093
:1024E60066F103C067F164C158F165C159F166C16F
:1024F6005AF167C15BF164C100F065C101F066C1C4
:1025060002F067C103F058EC0DF0C5EC05F000C011
:1025160004F001C005F002C006F003C007F064C174
:1025260000F065C101F066C102F067C103F00BEC73
:102536000EF0000E046E000E056E000E066E7E0E88
:10254600076EF1EC08F0000ED8B0010E006E0052D6
:102556001AE058C100F059C101F05AC102F05BC13E
:1025660003F0000E046E000E056E000E066E7E0E63
:10257600076ED3EC02F000C058F101C059F102C059
:102586005AF103C05BF158C100F059C101F05AC1BC
:1025960002F05BC103F058EC0DF001015351010F3D
:1025A600096E0A6A000E0A2209C004F00AC005F084
:1025B600000E0ABEFF0E066E076E04360490053640
:1025C6000636073604360490053606360736570EA5
:1025D6000424F66E490E0520F76E000E0620F86EEE
:1025E6000900F5CF05F00900F5CF06F00900F5CF93
:1025F60007F00900F5CF08F00850035C08E1075022
:10260600025C05E10650015C02E10550005C1EE338
:10261600010158C100F059C101F05AC102F05BC175
:1026260003F0CD0E046ECC0E056E4C0E066E7B0EC0
:10263600076EF4EC01F000C058F101C059F102C078
:102646005AF103C05BF15C4B5D2B5AD058C100F0C8
:1026560059C101F05AC102F05BC103F058EC0DF00C
:1026660053C104F0000E056E066E076E0436049024
:10267600053606360736043604900536063607361E
:10268600570E0424F66E490E0520F76E000E06203E
:10269600F86E0900F5CF05F00900F5CF06F0090040
:1026A600F5CF07F00900F5CF08F00850035C08E104
:1026B6000750025C05E10650015C02E10550005C32
:1026C6001FE2010158C100F059C101F05AC102F0E0
:1026D6005BC103F0000E046E000E056E200E066E42
:1026E600820E076EF4EC01F000C058F101C059F1FA
:1026F60002C05AF103C05BF1010E5C5F000E5D5B28
:10270600010157A393D057B791D0800E000A006EEF
:10271600800E5219005C02E151510A0804E20A0EC9
:10272600516F000E526F58C100F059C101F05AC1E5
:1027360002F05BC103F058EC0DF000C05EF101C081
:102746005FF102C060F103C061F15E515F1160117B
:10275600611142E00A0E046E000E056E066E076EEB
:102766005EC100F05FC101F060C102F061C103F01B
:1027760000EC06F008C000F009C001F00AC002F043
:102786000BC003F0000E046E031808E10450021893
:1027960005E10450011802E10050000A1DE1010E96
:1027A600515F000E525B0A0E046E000E056E066E39
:1027B600076E5EC100F05FC101F060C102F061C149
:1027C60003F000EC06F000C05EF101C05FF102C04C
:1027D60060F103C061F1B9D7800E5219006E800E08
:1027E600005C02E15351515D21E25151535D6A6F24
:1027F600BCEC09F000C004F001C005F002C006F010
:1028060003C007F058C100F059C101F05AC102F0E7
:102816005BC103F09AEC0CF000C058F101C059F10D
:1028260002C05AF103C05BF151C153F1050E01011B
:102836005125006E000E5221016E0050545F01506A
:10284600555B5151521103E157B701D004D0010E27
:10285600545F000E555B030E5615006E57C101F00E
:10286600000E01160050011004E0010E545F000E28
:10287600555B56A539D056A312D056A103D02D0EBE
:10288600496F02D02B0E496F42C1E1FF43C1E2FFFF
:1028960049C1E6FF424B432B624B632B0CD056A13A
:1028A6000AD042C1E1FF43C1E2FF200EE66E424B71
:1028B600432B624B632B800E006E800E5519005C15
:1028C60002E1545100080FE242C1E1FF43C1E2FFB9
:1028D600300EE66E424B432B624B632B010E545F68
:1028E600000E555BE8D73AD056B718D0800E006E6A
:1028F600800E5519005C02E1545100080FE242C1F6
:10290600E1FF43C1E2FF200EE66E424B432B624BD2
:10291600632B010E545F000E555BE8D756A312D009
:1029260056A103D02D0E4A6F02D02B0E4A6F42C11C
:10293600E1FF43C1E2FF4AC1E6FF424B432B624B34
:10294600632B0CD056A10AD042C1E1FF43C1E2FF7E
:10295600200EE66E424B432B624B632B58C100F0B0
:1029660059C101F05AC102F05BC103F058EC0DF0F9
:1029760000C05EF101C05FF102C060F103C061F109
:1029860053C100F0000E016E026E036E0036009019
:10299600013602360336003600900136023603361B
:1029A600570E0024F66E490E0120F76E000E022027
:1029B600F86E0900F5CF04F00900F5CF05F009001F
:1029C600F5CF06F00900F5CF07F05EC100F05FC154
:1029D60001F060C102F061C103F000EC06F0300EB8
:1029E600002642C1E1FF43C1E2FF00C0E6FF424BC1
:1029F600432B624B632B5151521103E157B701D060
:102A06006FD042C1E1FF43C1E2FF2E0EE66E424B9C
:102A1600432B624B632B5351515F000E525B535352
:102A26004DE0530753C100F0000E016E026E036EB7
:102A36000036009001360236033600360090013625
:102A460002360336570E0024F66E490E0120F76E45
:102A5600000E0220F86E0900F5CF04F00900F5CF4C
:102A660005F00900F5CF06F00900F5CF07F05EC1C5
:102A760000F05FC101F060C102F061C103F000EC3B
:102A860006F00A0E046E000E056E066E076E00EC6A
:102A960006F008C000F009C001F00AC002F00BC041
:102AA60003F0300E002642C1E1FF43C1E2FF00C041
:102AB600E6FF424B432B624B632BB1D75151521168
:102AC6000FE042C1E1FF43C1E2FF300EE66E424B2A
:102AD600432B624B632B010E515F000E525BEED708
:102AE60056AB0BD042C1E1FF43C1E2FF450EE66E95
:102AF600424B432B624B632B0AD042C1E1FF43C1D9
:102B0600E2FF650EE66E424B432B624B632B800E53
:102B16005D19006E800E005C02E1000E5C5D11E244
:102B26005C5100085C6F5D51000E5D5742C1E1FFCC
:102B360043C1E2FF2D0EE66E424B432B624B632BE5
:102B46000AD042C1E1FF43C1E2FF2B0EE66E424BC3
:102B5600432B624B632B0A0E046E000E056E5CC19E
:102B660000F05DC101F058EC09F0300E002642C1BC
:102B7600E1FF43C1E2FF00C0E6FF0101424B432BE8
:102B8600624B632B0A0E046E000E056E5CC100F0EC
:102B96005DC101F058EC09F008C000F009C001F071
:102BA600300E002642C1E1FF43C1E2FF00C0E6FF4E
:102BB6000101424B432B624B632B56A71AD0800E62
:102BC600006E800E5519005C02E15451000811E2B6
:102BD60042C1E1FF43C1E2FF200EE66E424B432BAA
:102BE600624B632B010E545F000E555B5451551119
:102BF600EFE120EF0EF057A3F3D0800E5D19006EC3
:102C0600800E005C02E1000E5C5D0AE2010E5C5D76
:102C1600006E000E5D59016E0050515F0150525B0F
:102C260058C100F059C101F05AC102F05BC103F06E
:102C360058EC0DF000C05EF101C05FF102C060F11A
:102C460003C061F1010E536F53510A0A34E053C1B8
:102C560000F0000E016E026E036E00360090013623
:102C66000236033600360090013602360336570E1A
:102C76000024F66E490E0120F76E000E0220F86E53
:102C86000900F5CF01F00900F5CF02F00900F5CFF4
:102C960003F00900F5CF04F00450615D08E103502C
:102CA600605D05E102505F5D02E101505E5D01E29B
:102CB60002D0532BC9D75351515D686F000E52593C
:102CC600696F68C151F169C152F15EC100F05FC11F
:102CD60001F060C102F061C103F0C5EC05F000C06F
:102CE60004F001C005F002C006F003C007F058C1A9
:102CF60000F059C101F05AC102F05BC103F00BECC0
:102D06000EF000C064F101C065F102C066F103C0B7
:102D160067F168C16AF1BCEC09F064C104F065C1F1
:102D260005F066C106F067C107F0F4EC01F0000E8D
:102D3600046E000E056E000E066E7E0E076ED3EC58
:102D460002F058EC0DF000C05EF101C05FF102C068
:102D560060F103C061F15151521142E00A0E046E56
:102D6600000E056E066E076E5EC100F05FC101F0D3
:102D760060C102F061C103F000EC06F008C000F08B
:102D860009C001F00AC002F00BC003F0000E046E89
:102D9600031808E10450021805E10450011802E185
:102DA6000050000A1DE10A0E046E000E056E066E46
:102DB600076E5EC100F05FC101F060C102F061C143
:102DC60003F000EC06F000C05EF101C05FF102C046
:102DD60060F103C061F1010E515F000E525BBBD77B
:102DE600800E006E800E5219005C02E151510C08F3
:102DF60016E351C16AF176EC07F058C104F059C1E7
:102E060005F05AC106F05BC107F0D3EC02F000C032
:102E160058F101C059F102C05AF103C05BF158C123
:102E260000F059C101F05AC102F05BC103F0046A17
:102E3600056A066A076AF4EC0DF0000ED8A4010EC6
:102E4600006E0052D8B477D058C100F059C101F0D5
:102E56005AC102F05BC103F058EC0DF0000E046E8F
:102E6600031808E10450021805E10450011802E1B4
:102E76000050000A60E1800E006E800E5D19005C55
:102E860002E15C51010857E25CC16AF1BCEC09F051
:102E960000C004F001C005F002C006F003C007F050
:102EA60058C100F059C101F05AC102F05BC103F0EC
:102EB6009AEC0CF05F0E046E700E056E090E066E2F
:102EC600810E076EF1EC08F0010ED8B0000E006E10
:102ED600005206E0090E01015C5F000E5D5B05D045
:102EE6000101080E5C5F000E5D5B5CC16AF1BCEC23
:102EF60009F000C004F001C005F002C006F003C0EE
:102F060007F058C100F059C101F05AC102F05BC187
:102F160003F09AEC0CF058EC0DF000C05EF101C025
:102F26005FF102C060F103C061F10101586B596B9A
:102F36005A6B5B6B38D058C100F059C101F05AC1C9
:102F460002F05BC103F058EC0DF000C05EF101C069
:102F56005FF102C060F103C061F15EC100F05FC1C4
:102F660001F060C102F061C103F0C5EC05F000C0DC
:102F760004F001C005F002C006F003C007F058C116
:102F860000F059C101F05AC102F05BC103F00BEC2D
:102F96000EF000C058F101C059F102C05AF103C049
:102FA6005BF15C6B5D6B010E536F53510A0A34E0A3
:102FB60053C100F0000E016E026E036E00360090E3
:102FC60001360236033600360090013602360336E5
:102FD600570E0024F66E490E0120F76E000E0220F1
:102FE600F86E0900F5CF01F00900F5CF02F00900EF
:102FF600F5CF03F00900F5CF04F00450615D08E158
:103006000350605D05E102505F5D02E101505E5DC7
:1030160001E202D0532BC9D753515125006E000E41
:103026005221016E5C5100265D5101220050545F11
:103036000150555B57B704D05151521101E104D0EC
:10304600010E545F000E555B030E5615006E57C1F8
:1030560001F0000E01160050011004E0010E545F4D
:10306600000E555B56A539D056A312D056A103D0F3
:103076002D0E4B6F02D02B0E4B6F42C1E1FF43C1A9
:10308600E2FF4BC1E6FF424B432B624B632B0CD056
:1030960056A10AD042C1E1FF43C1E2FF200EE66E0F
:1030A600424B432B624B632B800E006E800E5519EC
:1030B600005C02E1545100080FE242C1E1FF43C146
:1030C600E2FF300EE66E424B432B624B632B010E42
:1030D600545F000E555BE8D73AD056B718D0800E2D
:1030E600006E800E5519005C02E1545100080FE293
:1030F60042C1E1FF43C1E2FF200EE66E424B432B85
:10310600624B632B010E545F000E555BE8D756A346
:1031160012D056A103D02D0E4C6F02D02B0E4C6F41
:1031260042C1E1FF43C1E2FF4CC1E6FF424B432BE4
:10313600624B632B0CD056A10AD042C1E1FF43C1BA
:10314600E2FF200EE66E424B432B624B632B53C1CC
:1031560000F0530700524CE053C100F0000E016E20
:10316600026E036E003600900136023603360036D4
:103176000090013602360336570E0024F66E490ECD
:103186000120F76E000E0220F86E0900F5CF04F05C
:103196000900F5CF05F00900F5CF06F00900F5CFD7
:1031A60007F05EC100F05FC101F060C102F061C1CD
:1031B60003F000EC06F00A0E046E000E056E066EB5
:1031C600076E00EC06F008C000F009C001F00AC066
:1031D60002F00BC003F0300E002642C1E1FF43C1EE
:1031E600E2FF00C0E6FF424B432B624B632BAFD797
:1031F600800E006E800E5D19005C02E15C510008D5
:103206000FE242C1E1FF43C1E2FF300EE66E424BE0
:10321600432B624B632B010E5C5F000E5D5BE8D7B0
:10322600800E000A006E800E5219005C02E15151B8
:10323600080803E2080E536F02D051C153F15351EF
:10324600515F000E525B535303E157B701D00AD0CA
:1032560042C1E1FF43C1E2FF2E0EE66E424B432B15
:10326600624B632B53C16AF1BCEC09F058C104F000
:1032760059C105F05AC106F05BC107F0F4EC01F044
:103286002DEC05F000C05EF101C05FF102C060F1F7
:1032960003C061F153534DE0530753C100F0000ED4
:1032A600016E026E036E003600900136023603365A
:1032B60000360090013602360336570E0024F66EAD
:1032C600490E0120F76E000E0220F86E0900F5CFB8
:1032D60004F00900F5CF05F00900F5CF06F0090066
:1032E600F5CF07F05EC100F05FC101F060C102F0EA
:1032F60061C103F000EC06F00A0E046E000E056EC6
:10330600066E076E00EC06F008C000F009C001F07A
:103316000AC002F00BC003F0300E002642C1E1FFE6
:1033260043C1E2FF00C0E6FF424B432B624B632BD7
:10333600B1D7515152110FE042C1E1FF43C1E2FF43
:10334600300EE66E424B432B624B632B010E515FF0
:10335600000E525BEED756A71AD0800E006E800E76
:103366005519005C02E15451000811E242C1E1FF27
:1033760043C1E2FF200EE66E424B432B624B632BAA
:10338600010E545F000E555B54515511EFE120EFCD
:103396000EF0C00E5615016E57C102F0000E021651
:1033A600000E021802E1000E0118D8A480D056A91A
:1033B60027D047C1E9FF48C1EAFFEECF00F0EECFC4
:1033C60001F000C0E9FF01C0EAFFEECF5EF1EECFEB
:1033D6005FF1EECF60F1EECF61F147C1E9FF48C181
:1033E600EAFF040EEE24006E000EEE20016E47C1C9
:1033F600E1FF48C1E2FF00C0E6FF01C0E6FF2FD0B3
:1034060047C1E9FF48C1EAFFEECF00F0EECF01F079
:1034160000C0E9FF01C0EAFFEECF00F0EECF01F0F9
:10342600000E01BEFF0E026E036E00C05EF101C00B
:103436005FF102C060F103C061F147C1E9FF48C115
:10344600EAFF020EEE24006E000EEE20016E47C16A
:10345600E1FF48C1E2FF00C0E6FF01C0E6FF800EC3
:103466006119006E800E005C08E1000E605D05E1EA
:10347600000E5F5D02E1000E5E5D18E2030E56135C
:10348600000E5713006A016A026A036A5E51005E03
:103496005F51015A6051025A6151035A00C05EF1F0
:1034A60001C05FF102C060F103C061F14ED056A9C0
:1034B60027D047C1E9FF48C1EAFFEECF00F0EECFC3
:1034C60001F000C0E9FF01C0EAFFEECF5EF1EECFEA
:1034D6005FF1EECF60F1EECF61F147C1E9FF48C180
:1034E600EAFF040EEE24006E000EEE20016E47C1C8
:1034F600E1FF48C1E2FF00C0E6FF01C0E6FF25D0BC
:1035060047C1E9FF48C1EAFFEECF00F0EECF01F078
:1035160000C0E9FF01C0EAFFEECF5EF1EECF5FF13A
:10352600000E606F616F47C1E9FF48C1EAFF020EF6
:10353600EE24006E000EEE20016E47C1E1FF48C189
:10354600E2FF00C0E6FF01C0E6FF000E521902E1ED
:10355600000E51190FE1000E006E611908E10050CE
:10356600601905E100505F1902E15E51000A02E1AF
:10357600514B522BC00E5615006E00C005F0AED052
:10358600010E536F53510A0A34E053C100F0000E86
:10359600016E026E036E0036009001360236033667
:1035A60000360090013602360336570E0024F66EBA
:1035B600490E0120F76E000E0220F86E0900F5CFC5
:1035C60001F00900F5CF02F00900F5CF03F009007C
:1035D600F5CF04F00450615D08E10350605D05E13C
:1035E60002505F5D02E101505E5D01E202D0532BA5
:1035F600C9D782D0010E536F5351080A34E053C124
:1036060000F0000E016E026E036E00360090013669
:103616000236033600360090013602360336A50E12
:103626000024F66E490E0120F76E000E0220F86E99
:103636000900F5CF01F00900F5CF02F00900F5CF3A
:1036460003F00900F5CF04F00450615D08E1035072
:10365600605D05E102505F5D02E101505E5D01E2E1
:1036660002D0532BC9D748D0010E536F53510C0AC1
:1036760034E053C100F0000E016E026E036E003698
:1036860000900136023603360036009001360236C7
:1036960003369A0E0024F66E480E0120F76E000ED1
:1036A6000220F86E0900F5CF01F00900F5CF02F00F
:1036B6000900F5CF03F00900F5CF04F00450615D71
:1036C60008E10350605D05E102505F5D02E10150D3
:1036D6005E5D01E202D0532BC9D70ED00550000A19
:1036E600D8B44ED70550C00AD8B44AD70550800A78
:1036F60081E00550400AB8E0800E006E800E521937
:10370600005C02E15151535D03E251C153F10DD00A
:10371600800E5219006E800E005C02E15351515D1D
:1037260004E253C151F1000E526F545155110EE08F
:10373600030E5615006E57C101F0000E011600501B
:10374600011004E0010E545F000E555B800E521905
:10375600006E800E5519005C02E15451515D05E280
:103766005151545F5251555B02D0546B556BC40E88
:103776005615016E5751080B026E0250080A02E1F7
:10378600400E011808E15451551104E0010E545F32
:10379600000E555B1CD0C00E5615016E5751080B16
:1037A600026E0250080A02E1800E011810E1800E36
:1037B600006E800E5519005C02E15451020805E2C4
:1037C600020E545F000E555B02D0546B556B56A526
:1037D6005DD056A312D056A103D02D0E4D6F02D048
:1037E6002B0E4D6F42C1E1FF43C1E2FF4DC1E6FF23
:1037F600424B432B624B632B34D056A10BD042C1B4
:10380600E1FF43C1E2FF200EE66E424B432B624BC3
:10381600632B27D0C00E5615016E5751080B026E4A
:103826000250080A02E1800E01181BE142C1E1FFC5
:1038360043C1E2FF300EE66E424B432B624B632BD5
:1038460056AB03D0580E4E6F02D0780E4E6F42C163
:10385600E1FF43C1E2FF4EC1E6FF424B432B624B01
:10386600632B5451551111E042C1E1FF43C1E2FF00
:10387600300EE66E424B432B624B632B010E545FB8
:10388600000E555B54515511EFE174D0545155114A
:1038960013E056B711D042C1E1FF43C1E2FF200E4B
:1038A600E66E424B432B624B632B010E545F000EB8
:1038B600555B54515511EFE156A312D056A103D0D2
:1038C6002D0E4F6F02D02B0E4F6F42C1E1FF43C149
:1038D600E2FF4FC1E6FF424B432B624B632B0CD0FA
:1038E60056A10AD042C1E1FF43C1E2FF200EE66EB7
:1038F600424B432B624B632BC00E5615016E57513C
:10390600080B026E0250080A02E1400E01180BE194
:1039160042C1E1FF43C1E2FF300EE66E424B432B4C
:10392600624B632B27D0C00E5615016E5751080BFC
:10393600026E0250080A02E1800E01181BE142C124
:10394600E1FF43C1E2FF300EE66E424B432B624B72
:10395600632B56AB03D0580E506F02D0780E506FC3
:1039660042C1E1FF43C1E2FF50C1E6FF424B432B98
:10397600624B632B800E006E800E5219005C02E1D2
:103986005151535D0BE242C1E1FF43C1E2FF300EEC
:10399600E66E424B432B624B632BECD751C100F0D2
:1039A60052C101F0010E515F000E525B0050011032
:1039B600D8B42AD1C00E5615006E00C064F10AD1E3
:1039C60051C100F052C101F0000E52BFFF0E026E4F
:1039D600036E00360090013602360336003600903C
:1039E600013602360336570E0024F66E490E0120C4
:1039F600F76E000E0220F86E0900F5CF04F00900FC
:103A0600F5CF05F00900F5CF06F00900F5CF07F070
:103A16005EC100F05FC101F060C102F061C103F058
:103A260000EC06F00A0E046E000E056E066E076EBA
:103A360000EC06F008C000F009C001F00AC002F070
:103A46000BC003F0300E0024536FD3D056AB45D0D5
:103A560051C100F052C101F0000E52BFFF0E026EBE
:103A6600036E0036009001360236033600360090AB
:103A7600013602360336A50E0024F66E490E0120E5
:103A8600F76E000E0220F86E0900F5CF04F009006B
:103A9600F5CF05F00900F5CF06F00900F5CF07F0E0
:103AA6005EC100F05FC101F060C102F061C103F0C8
:103AB60000EC06F00F0E0016000E01160216031695
:103AC600290E0024F66E4A0E0120F76E000E022023
:103AD600F86E0900F5CF53F144D051C100F052C140
:103AE60001F0000E52BFFF0E026E036E003600900C
:103AF60001360236033600360090013602360336AA
:103B0600A50E0024F66E490E0120F76E000E022067
:103B1600F86E0900F5CF04F00900F5CF05F00900AD
:103B2600F5CF06F00900F5CF07F05EC100F05FC1E2
:103B360001F060C102F061C103F000EC06F00F0E67
:103B46000016000E0116021603163A0E0024F66E33
:103B56004A0E0120F76E000E0220F86E0900F5CF1E
:103B660053F147D051C100F052C101F0000E52BFCF
:103B7600FF0E026E036E00360090013602360336E3
:103B8600003600900136023603369A0E0024F66E91
:103B9600480E0120F76E000E0220F86E0900F5CFE0
:103BA60004F00900F5CF05F00900F5CF06F009008D
:103BB600F5CF07F05EC100F05FC101F060C102F011
:103BC60061C103F000EC06F0070E0014536F300ECF
:103BD60053270FD06451000AD8B4F2D66451C00AF4
:103BE600D8B4EED66451800AD8B430D76451400AAE
:103BF600B9E042C1E1FF43C1E2FF53C1E6FF424BD8
:103C0600432B624B632BCAD656A71AD0800E006E82
:103C1600800E5519005C02E15451000811E242C1C0
:103C2600E1FF43C1E2FF200EE66E424B432B624B9F
:103C3600632B010E545F000E555B54515511EFE195
:0E3C460020EF0EF062C100F063C101F0120029
:103C540042C102F043C103F002C000F003C001F00E
:103C6400024A032A00C0E9FF01C0EAFFEE5201E064
:103C7400F3D701014251025C006E43510358016EB7
:0A3C8400010E005E000E015A12004E
:0A3C8E001D0E0D6E0D2EFED7120064
:0E3C9800ACB202D00000FCD742C1ADFF12005A
:103CA60042C1E9FF43C1EAFFEE500101441905E1B3
:103CB60042C100F043C101F010D042C100F043C13F
:103CC60001F0424B432B00C0E9FF01C0EAFFEECFF3
:0C3CD60000F00052E5E1006A016A1200F3
:103CE20046C100F001014607005228E042C1E9FF47
:103CF20043C1EAFFEE50000A0CE042C1E9FF43C1B2
:103D0200EAFF44C1D9FF45C1DAFFEE50DE1801E1F6
:103D12000FD042C1E9FF43C1EAFF44C1D9FF45C107
:103D2200DAFFDE50EE5C006E016A000E015A08D026
:103D32000101424B432B444B452BD2D7006A016A07
:023D420012006D
:103D4400800ED56E630ED76EC00ED66EF29A120038
:103D5400010EB16EA192F00EB36E600EB26EA0822F
:0C3D6400C00EF26EB190B19EB19C120036
:103D7000CD6A9E90F00ECF6E600ECE6E9D80C00E0E
:0A3D8000F26ECD90CD9ECD9C120096
:103D8A00340E0101406F010E416F2FC142F130C163
:103D9A0043F131C144F132C145F133C146F1400E1C
:103DAA00476F010E486F1BEC0EF000C03EF101C0D8
:103DBA003FF100502F25E16E01503021E26EE66A94
:0A3DCA003EC100F03FC101F01200FD
:103DD400000E0101301902E1000E2F1934E02FC149
:103DE400E9FF30C1EAFFEE522EE031C142F132C1A7
:103DF40043F12EDF00C046F12FC142F130C143F13F
:103E040031C144F132C145F16ADF000E011802E10B
:103E1400000E001805E12FC100F030C101F015D0EB
:103E2400010E01012F25426F000E3021436F31C175
:103E3400E9FF32C1EAFFEECF44F133DF00C02FF1D6
:0C3E440001C030F1C5D7006A016A12000D
:103E5000150E0B6E4B0E0C6EBE0E0D6E0D2EFED79C
:0C3E60000C2EFCD70B2EFAD7000012002D
:103E6C00C26A431C006E0050C1160F0EC012C08EE9
:103E7C002FC100F000360090003600900050C212A6
:103E8C00C280FFDEC282C2A201D0FDD7C4CF01F036
:103E9C00006A00C030F101C031F1C3500012000EB5
:103EAC00011200C030F101C031F1C290000E0014BB
:103EBC00026E0150800B036E000E031802E1000E1F
:103ECC00021803E00101306B316B30C100F031C1DD
:043EDC0001F01200DF
:103EE000FF0E816E830E936E0F01396BF19EFF0EF4
:103EF000616E9392939493968A928A948A96796A41
:103F0000786A806A386B3881388338850F0E926EF4
:103F1000806A92988998826A3A6B946A9496948897
:083F2000948E949C606A12006B
:103F2800980E0001B96F3C0EBA6F420EBB6F010EBE
:103F3800BC6FFF0EC96FFF0ECA6F000ECB6F000E6D
:103F4800CC6FFF0ECD6FFF0ECE6F000ECF6F000E41
:103F5800D06FFF0EC56FFF0EC66F000EC76F000E45
:103F6800C86FAC8A900EAB6E948E949C9EAA03D0B8
:083F7800AECF00F0FBD71200F0
:103F80002FC1E9FF30C1EAFFEECF31F1000E010190
:103F9000326F000E326F000E321902E1200E31191D
:103FA00007E0000E321902E1090E311901E003D0D9
:103FB0002F4B302BE5D7336B346B356B366B000EE4
:103FC000321902E12D0E311905E1354B362B2F4BFD
:103FD000302B08D0000E321902E12B0E311902E10C
:103FE0002F4B302B2FC1E9FF30C1EAFFEECF31F16B
:103FF000000E326F000E326F31C16AF10FEC0EF01D
:10400000005219E033C100F034C101F00A0E046E11
:10401000000E056ED8EC05F0300E315D026E000E1C
:104020003259036E02500024336F03500120346F65
:104030002F4B302BD7D73551361108E033510008BC
:10404000006E34C101F0000E015604D033C100F0FF
:0640500034C101F0120072
:104056000900F5CFE6FF0006FBE10106F9E11200D3
:10406600FF0E0001BD6FFF0EBE6FFF0EBF6FFF0E8E
:10407600C06FC26A431C006E0050C1160F0EC012FC
:06408600C08EC280120092
:10408C002FC1E9FF30C1EAFFEE520BE02FC1E9FF6F
:10409C0030C1EAFFEECF42F1F9DD01012F4B302B9D
:0440AC00EFD7120038
:1040B0000D0E0101426FF0DD0A0E0101426FECDDD1
:0240C0001200EC
:1040C2002FC1F6FF30C1F7FF31C1F8FF0900F5CF6C
:1040D20000F0005211E02FC1F6FF30C1F7FF31C1ED
:1040E200F8FF0900F5CF42F1D6DD010E01012F27BD
:0A40F200000E30233123E4D7120042
:1040FC0047EC25F09B6A720ED36ED26AD3B401D012
:10410C00FDD7E8DE89880001B56BB66BB76BB86B71
:10411C00A56BA66BA5C0B3F0A6C0B4F0550EA76FE7
:10412C00000EA86F550EA76F000EA86FB886B06A68
:10413C00CF0EAF6EAC84F2DE030E0B6E080E0C6E5F
:10414C00770E0D6E0D2EFED70C2EFCD70B2EFAD73C
:10415C000C0E0101426F9ADDA5DF0B0E0B6E260EC5
:10416C000C6E5D0E0D6E0D2EFED70C2EFCD70B2E8D
:10417C00FAD700000000516A526A536A546A550E0D
:10418C000001A76F000EA86FB16BB26B800EB21955
:10419C00006E800E005C02E10B0EB15D27E2030E97
:1041AC00006E000E016EB1C004F0B2C005F0D8EC88
:1041BC0005F01B0E0024E96E000E0120EA6EEECF16
:1041CC002FF1EECF30F1EECF31F175DF030E0B6E28
:1041DC00080E0C6E770E0D6E0D2EFED70C2EFCD726
:1041EC000B2EFAD70001B14BB22BD0D78998516A5C
:1041FC00526A33DFAD6BAE6BAF6BB06B516A526A08
:10420C00A96BAA6BD08EF28C9D8AF1849F809F82C1
:10421C00A282F28EAB6BAC6B7C0E01012F6F460E43
:10422C00306F000E316F47DF5F0E0001D86FF00E5C
:10423C00D96F8F0EDA6FE80EDB6FA7C02FF1A8C015
:10424C0030F18E0E0101316F470E326F000E336F5D
:10425C0051C034F152C035F1D6C036F1D7C037F168
:10426C005F0E386FF00E396FD2C03AF1D3C03BF10C
:10427C008F0E3C6FE80E3D6F82DDA7C02FF1A8C0FA
:10428C0030F1FEDE0FDF0001D46BD56B5DDD6ADD36
:10429C0053DDF28AD58E01012F6BE2DD00C0D6F022
:1042AC0001C0D7F00150030802E10050E80805E214
:1042BC00E80E0001D66F030ED76F010E01012F6FB0
:1042CC00CFDD00C0D2F001C0D3F00150030802E1F1
:1042DC000050E80805E2E80E0001D26F030ED36F20
:1042EC000001550EA76F000EA86FA7C02FF1A8C034
:1042FC0030F14F0E0101316F470E326F000E336FEC
:10430C0051C034F152C035F1D6C036F1D7C037F1B7
:10431C00D8C038F1D9C039F1D2C03AF1D3C03BF191
:10432C00DAC03CF1DBC03DF12ADDA7C02FF1A8C0FB
:10433C0030F1A6DEB7DE5050010A37E1E80E00017D
:10434C00D625036E030ED721046E03C000F004C003
:10435C0001F000360090013600360090013600C0A6
:10436C00A9F001C0AAF00050FF08D86F01C0D9F025
:10437C00FF0ED957E80ED225036E030ED321046E1F
:10438C0003C000F004C001F0003600900136003686
:10439C000090013600C0A9F001C0AAF00050FF083F
:1043AC00DA6F01C0DBF0FF0EDB570001B76BB86BA7
:1043BC00B56BB66B9D8ADF6BDE6BDC6BDD6B42DD48
:1043CC0041DD000EB81902E1010EB719D8A424D1B1
:1043DC00EB6B710E01012F6F4A0E306F000E316FB7
:1043EC006ADEDF0E01012F6F000E306F49DEDF0E2B
:1043FC0001012F6F000E306F4B0E316F000E326FBC
:10440C00E3DC00C0D4F001C0D5F0000E026E015008
:10441C00025C02E100500008D8B0C6D0D4C042F112
:10442C00D5C043F111DC00C0A9F001C0AAF0000E08
:10443C00011802E10A0E0018D8A4B2D0536A546ACB
:10444C00040E0001D425E96E000ED521EA6EEECFE4
:10445C00D1F0B16BB26B800EB219006E800E005CA5
:10446C0002E1040EB15D18E2060ED425006E000EBA
:10447C00D521016EB1510024E96EB2510120EA6ED2
:10448C00EECF6AF10FEC0EF000505326000E5422C2
:10449C000001B14BB22BDFD7060EA95D016E000EE9
:1044AC00AA59026E5450021802E101505318D8A4B4
:1044BC006FD0060ED42501012F6F000E0001D521FF
:1044CC000101306F57DD00C0A9F001C0AAF0800EC9
:1044DC000118026E800E030A025C02E1E80E005C19
:1044EC004EE3800E070A006E800E0001AA19005CD4
:1044FC0002E1A951D00843E3840E01012F6F4A0E4B
:10450C00306F000E316FD7DD0001A937A991AA37A2
:10451C00A937A991AA372AD0A951FF08D86FAAC0E8
:10452C00D9F0FF0ED957780E01012F6F4A0E306F5C
:10453C00000E316FC0DD22D00001A951FF08DA6FE7
:10454C00AAC0DBF0FF0EDB57690E01012F6F4A0E7C
:10455C00306F000E316FAFDD11D04B0E01012F6F9C
:10456C004A0E306F000E316FA6DD08D00001D1511C
:10457C00310AD2E0D151320ADFE0EFD708D0E50E94
:10458C0001012F6F490E306F000E316F94DD08D092
:10459C00FC0E01012F6F490E306F000E316F8BDD59
:1045AC000001D46BD56B7EDDDF0E01012F6F000E89
:1045BC00306F440E316F000E326F06DC00C0D4F049
:1045CC0001C0D5F0000E026E0150025C02E10050F9
:1045DC00000821E2060E0001D425E96E000ED5215B
:1045EC00EA6EEE50310A0BE1010E506E7F0E0101A6
:1045FC002F6F490E306F000E316F5DDD09D0506AA0
:10460C00CA0E01012F6F480E306F000E316F53DD53
:10461C000001D46BD56B46DD8978514A522A3BD6C2
:02462C00FFD7B6
:104A8E0010EE1BF0360E006E010E016ECC0EF66EA1
:0E4A9E00470EF76E000EF86E2BEC20F01200A3
:10462E0020536F75726365203A20426173655F3166
:10463E00384632364B32325F55415254315F327802
:10464E004144435F3278536572766F5F6D6F746568
:10465E0075725F54696D65725F315F325F335F32C1
:0E466E003032305F30345F32312E630D0A007F
:10467C000D0A20436F6E7369676E657320696E69EE
:10468C007469616C6973E9652061752064656D619D
:10469C0072726167652020436F6E7369676E653156
:1046AC003D316D532C20436F6E7369676E653220FC
:0B46BC003D20312C356D53200D0A000D
:1046C700204469726563746F72793A20433A5F4D8B
:1046D700696B726F435F4D657350726F6A65747370
:1046E7005F4D696B726F435C5F31384632364B32D0
:1046F700325F4364655F325F536572766F5F4D6FFC
:0847070074657572730D0A0060
:10470F002050726F6A6574203A20426173655F3181
:10471F00384632364B32325F55415254315F325F39
:10472F00536572766F5F4D6F746575725F3230329D
:10473F00305F30345F32312E6D637070690D0A0057
:10474F006A3D2025303564204541303D20253035E8
:10475F00642020436F6E7369676E65313D25303578
:10476F00752009204541313D2025303564202043F7
:0F477F006F6E7369676E65323D253035750900C1
:10478E006A3D2025303564204541303D20253035A9
:10479E00642020436F6E7369676E65313D253575F4
:1047AE002009204541313D20253035642020436FBE
:0E47BE006E7369676E65323D2535750D0A0014
:1047CC00C746000F47005B4A00FA4800134A006ACC
:1047DC004800C549002E46002A49007F4A00894AF4
:0147EC0000CC
:0747ED00286E756C6C2900B9
:0147F4000FB5
:0747F500504F5441523D00FA
:0547FC00434F4E530085
:0148010000B6
:104802000000007F000020820000488500007A88B6
:1048120000401C8C0050438F00247492809618969E
:1048220020BC3E99286B6E9CF90215A0EC782DC134
:04483200CAF249E29B
:104836000000007FCDCC4C7B0AD723786F1203751E
:1048460017B75171ACC5276EBD37066B95BF566756
:1048560077CC2B645F700961FFE65B5D08E53C3C45
:044866006042221B6F
:10486A0020506F727420486172642055415254314D
:10487A002031393230302C4E2C382C3120285243FA
:10488A00363D5458205243373D525829200D0A00CC
:10489A0001000000080000004000000000020000C3
:1048AA00001000000080000000000400000020004A
:1048BA0000000001000000080000004000000000A5
:1048CA000D0A204D6F646520736169736965206301
:1048DA006F6E7369676E65732076696120434C4118
:1048EA0056494554207465726D696E616C0D0A00F3
:1048FA0020436F6E666967203A2050313846323657
:10490A004B32325F464F53435F696E7465726E6510
:10491A005F31364D687A2E6366677363680D0A00E5
:10492A002075736573204C696272617279206164C3
:10493A00635F746F5F73696D696C695F666C6F61E1
:0D494A00745F7374722E6D636C200D0A0093
:10495700010000000A00000064000000E8030000F6
:1049670010270000A086010040420F0080969800A3
:0849770000E1F50500CA9A3BBE
:10497F000D0A204D6F64652073616973696520634B
:10498F006F6E7369676E65732076696120504F543F
:06499F004152730D0A00F5
:1049A50001000000100000000001000000100000E0
:1049B50000000100000010000000000100000010D0
:1049C50020496E6974205241302C312020617320BA
:1049D500416E616C6F6720496E707574200D0A0019
:1049E5006572726575722076616C6575722073618A
:0749F500697369650D0A00FA
:1049FC006572726575722076616C65757220736173
:074A0C00697369650D0A00E2
:104A130020464F534320696E7465726E65203136AC
:064A23004D487A0D0A0067
:104A290030313233343536373839414243444546DB
:014A3900007C
:104A3A00303132333435363738396162636465660A
:014A4A00006B
:104A4B00657272657572207361697369650D0A0011
:0E4A5B0020416C696D2E203D2035560D0A005D
:084A6900322E2E4F4B0D0A0006
:074A71000D0A5265633D00D0
:074A7800312E4F4B0D0A0027
:054A7F0020200D0A00DB
:054A8400434F4E5300FA
:044A8900200D0A00F2
:020000040030CA
:0D000100481E3CFFBF81FF0FC00FE00F4005
:00000001FF
